:1049A3000000090101240200000301FA0400FA05D2
:1049B30000020A0A5A0B000F0C00FA0D00030E0046
:1049C300030F0132100096120132130AFA14010286
:1049D30015000217010A18010A1905321A010A1BE8
:1049E300010A1C05321D010120010123011E2400BF
:1049F300642A00FA2B00FA2C50782D003C2E004636
:104A03002F001E3000643250783300003432FA3500
:104A13000164360164370150380A643C00643E0087
:104A23003C3F000140FFFF411450420A5A430AC869
:104A33004405324500784600FA4701224802034CF8
:104A430000FA4EFFFF500404510596520A32530BED
:104A530028540A96560102570546580002590A4639
:104A63005A32FA5B010A5C0A325E000A5F00FE6199
:104A7300FFFF6402106701036A0A3C6B00006C329B
:104A830096780132790132FAFAFA00000901012419
:104A93000200000301FA0400FA0500020A0A5A0B95
:104AA300000F0C00FA0D00030E00030F013210007B
:104AB30096120132130AFA14010215000017010AB3
:104AC30018010A1905321A010A1B010A1C05321DB5
:104AD300010120010123011E2400642A00FA2B0096
:104AE300FA2C50782D003C2E00462F001E30006417
:104AF3003250783300003432FA35016436016437BA
:104B03000150380A643C00643E003C3F000140FF12
:104B1300FF411450420A5A430AC8440532450078FB
:104B23004600FA4701224802024C00FA4EFFFF50AA
:104B33000404510596520A32530B28540A9656011F
:104B430001570546580001590A465A32FA5B010AD1
:104B53005C0A325E000A5F00FE61FFFF64021067B9
:104B630001036A0A3C6B00006C32967801327901CA
:104B730032FAFAFA0065006F00790083008D00971E
:104B830000A100AC00B600C000CA00D400DE00E8FB
:104B930000F2005B0063006A0072007A0082008901
:104BA3000091009900A100A800B000B800BF00C7A1
:104BB30000CF00D600DF00E600EE00F6004000461E
:104BC300004C00520059005F0065006B00710077D4
:104BD300007D00830089008F0095009C00A200A83F
:104BE30000AE00B400BA00C000C600CC00D200D9A9
:084BF30000DF00E500EB00F11A
:10009E00900082E0B4010385254F900082E0B40207
:1000AE00129000B8E08537F0A4FFAEF07408124E3F
:1000BE00778F4F900082E0B4030385394F90008212
:1000CE00E0B40403853F4F900082E0B40507E5409D
:1000DE00C39414F54F900082E0B4060385414F900F
:1000EE000082E0B4070385424F900082E0B408031B
:1000FE0085434F900082E0B40903853E4F90008304
:10010E00E0FE900084E0D39E405F900082E0B40455
:10011E0018900084E0C3954F5002D204900083E003
:10012E00D3954F4002C204803E900083E0C3954FAA
:10013E005009900084E0D3954F50028002D2049073
:10014E000083E0D3954F5009900084E0C3954F5043
:10015E0002C204900082E0B401099000C4E0D3957D
:10016E003950028002C204802A900083E0D3954F5A
:10017E004009900084E0C3954F40028002C2049073
:10018E000083E0C3954F4009900084E0D3954F4023
:10019E0002D2042285F94F85FA507E017F00E55088
:1001AE00124E85E54F2FFF50010E8E328F33900089
:1001BE0014E0FCA3E0FDEF2DFDEE3CFC8C348D3500
:1001CE002275A71085F94F85FA507E017F00E55004
:1001DE00124E85E54F2FFF50010E8E328F33900059
:1001EE00CBE0B40210AC55AD56EF2DFDEE3CFC8CC1
:1001FE00348D358016AE32AF33900014E0FCA3E0A0
:10020E00FDEF2DFDEE3CFC8C348D3522AE32AF333E
:10021E00740A8E048F05FF124E678C348D35AE3204
:10022E00AF33740A8E048F05FF124EA08C328D33BD
:10023E00E53345326013740AC39533FFE49532FEFD
:10024E008E328F337834124EE2E54FA834B8001553
:10025E00D395354010E54FC39535FFE49534FE8EAA
:10026E00348F358010E54F2424C39535FFE4953443
:10027E00FE8E348F35AE34AF3574236F4E600674F8
:10028E00246F4E701AAE34AF3574236F4E700575F1
:10029E004F018003754F027535227534008003754A
:1002AE004F0022900079E0B40104C2098002D20905
:1002BE0090007AE0B40104C20A8002D20A9000B71C
:1002CE00E075F0DCA4FFAEF0740A8E048F05FF1209
:1002DE004E6790079FECF0A3EDF0A2064016740354
:1002EE008C068D07124E857401124E7790079DEE87
:1002FE00F0A3EFF07E017F00900075E0124E859026
:10030E0000B8E08E048F05FF124E67740AFF124E7E
:10031E00678D389000C1E075F0DCA4FFAEF0740A72
:10032E008E048F05FF124E679007A3ECF0A3EDF03D
:10033E009000C3E060139000C3E0F5F0741684FFE4
:10034E007E00EF9007ABF0800674649007ABF090E0
:10035E0000A2E0B40B0874E3900064F080499000B2
:10036E00A2E0B419129000B8E0904B6212008CE437
:10037E0093900064F080309000A2E0B41E129000C2
:10038E00B8E0904B8012008CE493900064F08017DC
:10039E009000A2E0B428109000B8E0904BAA120092
:1003AE008CE493900064F0900040E0C394055022DA
:1003BE0074019000BBF09000BDE0B4020674019091
:1003CE0000BDF09000ADE0D39402400674029000A0
:1003DE00ADF09000D5E0B40117900020740FF0A39B
:1003EE0074FFF0900022E4F0A3F074029000D5F0B8
:1003FE009000D5E0B40341900022E0FEA3E0FF9010
:10040E000020E0FCA3E0FD124EDA7410124E85744B
:10041E0008124E77EF900061F0EF700674FF9000B7
:10042E0061F074009000D5F0900021E0900062F031
:10043E00900020E0900063F0900066E090002CF0B9
:10044E0090002CE0241290002DF090002DE0D3941B
:10045E0024400B90002DE0C3942490002DF09000CA
:10046E0030E4F090002CE06423600790002CE0B4A0
:10047E00242090002CE0B423067402900030F090FB
:10048E00002CE0B424069000307401F090002C741F
:10049E0001F0900031E4F090002DE06423600790AD
:1004AE00002DE0B4242090002DE0B42306740290B9
:1004BE000031F090002DE0B424069000317401F06C
:1004CE0090002D7401F0900066E0FE9000C9E02EC1
:1004DE00900033F0900033E0D39424400B9000331F
:1004EE00E0C39424900033F0900033E0B41206740D
:1004FE0013900033F0900033E0B424069000337470
:10050E0001F0900033E064116007900033E0B423F3
:10051E0006900033E014F0900033E0D39412400DB7
:10052E00900033E0C39412900034F0800A900033B0
:10053E00E02412900034F09000ACE090002EF09089
:10054E00002EE0B41206741390002EF090002EE0F0
:10055E00B41106741090002EF090002EE0D3941279
:10056E00400D90002EE0C3941290002FF0800A9060
:10057E00002EE0241290002FF022C293C294C2915A
:10058E00C292C287C290E5B554EFF5B5E5B554DF1A
:10059E00F5B5C296C295C2A0C297C2A2C2A1E5B5D8
:1005AE00547FF5B5E5B554BFF5B5E5B554FBF5B5D6
:1005BE00C20B7536469000AFE07005754802800399
:1005CE0075480390000874FFF0A374DCF09000905F
:1005DE00E090000EF8E4F0E8A3F0C210C21274C866
:1005EE00900024F074C8900028F075250075240042
:1005FE00C206756B00E54AB40903754A00753B00E7
:10060E00900016E4F0A3F0754B1E752700752600BA
:10061E00C20EC20F90079FE0FEA3E0FF7403124EBE
:10062E00857401124E7790079DEEF0A3EFF0C20392
:10063E0090000CE4F0A3F0C21D2285F94F85FA500C
:10064E007E017F00E550124E85E54F2FFF50010EC3
:10065E008E328F3390079FE0FCA3E0FDEF2DFDEE71
:10066E003CFC8C348D35E535F5FDE534F5FE220583
:10067E003C229000ADE0B403539000CBE0B4012EC9
:10068E00A2D8B34004C293C287A2D9B34004C29485
:10069E00C290A2DAB34008C291E5B554EFF5B5A207
:1006AE00DBB34008C292E5B554DFF5B5801CA2D885
:1006BE00B34002C293A2D9B34002C294A2DAB340AD
:1006CE0002C291A2DBB34002C2928012A2D8B34002
:1006DE0004C293C287A2D9B34004C294C290A2DCD2
:1006EE00B34004C296C29575D8402285A74E75A711
:1006FE0010A2D8B34002C287A2D9B34002C290A2C0
:10070E00DAB34006E5B554EFF5B5A2DBB34006E526
:10071E00B554DFF5B575D840854EA722900047E455
:10072E00936406600280FE74C89007A5F8E4F0E8B2
:10073E00A3F075B50075840175A70075FF8075EF80
:10074E0006900032E4F075C91075A70F75A1C77534
:10075E00A70075D90075CE0C75A70F75F1FE75F251
:10076E00FF75F30775F47875A4BA75A5FF75A6071E
:10077E0075AE0075AFFF75D48175D5FF75D6FF7553
:10078E00D7FF75A70075A20175A14775F80975D831
:10079E000075D90475DA0975DB0975DC0975DD0993
:1007AE0075DE0975D84075A71075D80075D9047512
:1007BE00DA0975DB0975DC0975DD0975D84075A791
:1007CE000075E60875E71075BC0175BE0475BD6C45
:1007DE0075BE0775BDA075BE0875BD0175BC0075EB
:1007EE00BB1875BC2075BA0875E88075D11375A74E
:1007FE000F75E10575E20075C740C293C294C291B0
:10080E00C292C287C290E5B554EFF5B5E5B554DF97
:10081E00F5B5C296C295C2A0C297C2A2C2A1E5B555
:10082E00547FF5B5E5B554BFF5B5E5B554FBF5B553
:10083E00759700759780740A124E577597C0E59795
:10084E005420700280F8758F0275A700D2AF75988C
:10085E000075A90C75A70F75AB4375ADFB75AC1E76
:10086E0075A71075C91875CA0075CB0075C80475C3
:10087E00A700758912758E04758C00758A00C2A941
:10088E00D28C758D00758B00D2ABD28E75D9447516
:10089E003100753000752D00752C007545007546BC
:1008AE0000C29974C8F509750800122DAF75B50010
:1008BE0074639007A5F8E4F0E8A3F012303B74647B
:1008CE00F509750800122DAFC21990004FE0B40162
:1008DE0008A2B54002D219802E90004FE0B402114A
:1008EE0075A70F75F30F75A700A2A34002D219804A
:1008FE001690004FE0B4030F75A70F75F31775A789
:10090E0000A2A44002D219A219B35003020A037422
:10091E00089007A5F8E4F0E8A3F0122F0A7464F526
:10092E0009750800122DAF74099007A5F8E4F0E8D8
:10093E00A3F0122F0A7464F509750800122DAF7416
:10094E000A9007A5F8E4F0E8A3F0122F0A7464F5F4
:10095E0009750800122DAF740B9007A5F8E4F0E8A6
:10096E00A3F0122F0A7464F509750800122DAF74E6
:10097E000C9007A5F8E4F0E8A3F0122F0A7464F5C2
:10098E0009750800122DAF740D9007A5F8E4F0E874
:10099E00A3F0122F0A7464F509750800122DAF74B6
:1009AE000E9007A5F8E4F0E8A3F0122F0A7464F590
:1009BE0009750800122DAF74029000AEF090004F32
:1009CE00E0900072F090004FE0B4010874009000C7
:1009DE007AF0801C90004FE0B4020874009000BDC5
:1009EE00F0800D90004FE0B4030674009000CAF042
:1009FE00D215020AE39007A5E4F0A304F0122F0A21
:100A0E007464F509750800122DAF74029007A5F8ED
:100A1E00E4F0E8A3F0122F0A7464F50975080012C9
:100A2E002DAF74039007A5F8E4F0E8A3F0122F0A97
:100A3E007464F509750800122DAF74049007A5F8BB
:100A4E00E4F0E8A3F0122F0A7464F5097508001299
:100A5E002DAF74059007A5F8E4F0E8A3F0122F0A65
:100A6E007464F509750800122DAF74069007A5F889
:100A7E00E4F0E8A3F0122F0A7464F5097508001269
:100A8E002DAF74079007A5F8E4F0E8A3F0122F0A33
:100A9E007464F509750800122DAF74019000AEF064
:100AAE0090004FE0900072F090004FE0B401087497
:100ABE000090007AF0801C90004FE0B402087400A1
:100ACE009000BDF0800D90004FE0B40306740090CE
:100ADE0000CAF0C2151231AF9000B8E07006740A69
:100AEE009000B8F0900064E0700674E3900064F03B
:100AFE001202B1E5B54401F5B5740690003EF074EE
:100B0E000190003FF07403900041F0740490004295
:100B1E00F07413900043F07405900044F090004080
:100B2E00E0B404067404900044F07403900045F0A1
:100B3E00740090004AF0740090004BF07401900025
:100B4E004CF0740090004DF074FF90004EF0743332
:100B5E0090013CF0743690013DF0742D90013EF002
:100B6E00743290013FF07420900140F07434900183
:100B7E0041F07443900142F07479900143F0746C2B
:100B8E00900144F07420900145F07442900146F0BB
:100B9E007465900147F07461900148F0746D900196
:100BAE0049F0747390014AF09000D4E0900061F027
:100BBE0090008BE0900062F090008CE0900063F06B
:100BCE00C210C21274C8900024F074C8900028F0AD
:100BDE00C20EC20FA2B6B39207A2B3B39208752586
:100BEE0000752400753646754B1E90005DE4F07559
:100BFE00261975276490000874FFF0A374DCF0C208
:100C0E000B754A00C20675290075280090000CE489
:100C1E00F0A3F0743A900765F074FD900766F075D6
:100C2E006C0090005EE4F0752B00752A00900010A9
:100C3E00E4F0A3F0900090E090000EF8E4F0E8A34A
:100C4E00F0900071E075F032A4FFAEF090001EEE51
:100C5E00F0A3EFF090079FE0FEA3E0FF7403124EA7
:100C6E00857401124E7790079DEEF0A3EFF0754953
:100C7E000190003AE4F0C21DC21A756B00753B007C
:100C8E00C20CC20DC21EC203754C00C204C205C204
:100C9E0016C217D21874FE900035F074FE9000360E
:100CAE00F0C21BD21C753700754300753900753DB7
:100CBE0032753E00753F00743C900038F075400070
:100CCE00743C900039F0754100754200900016E4B6
:100CDE00F0A3F0754400D2B2D2A4D2B0D2B1D2A356
:100CEE00D2A7D2A6D2A5D2B7900071E0D394FA4083
:100CFE000674FA900071F07E017F00900063E0129E
:100D0E004E85900062E02FFF50010E900020EEF015
:100D1E00A3EFF0EFD394FFEE940F4007900020E482
:100D2E00F0A3F0900061E0700674FF900061F09007
:100D3E0000AEE0D39402400674019000AEF0900035
:100D4E00AFE0700575480280037548039000B0E06F
:100D5E00D39401400674009000B0F09000B6E0C34A
:100D6E00940A5006740A9000B6F09000C0E0700627
:100D7E0074019000C0F09000C0E0B4FF0674FE90C5
:100D8E0000C0F09000C7E0D394FE400674FE9000C1
:100D9E00C7F074019000CDF074019000CEF0740095
:100DAE009000D0F074009000D5F0D29CD2EC75CFAC
:100DBE0001A298B350030211CAC298E546640460BA
:100DCE0006E59964FF6002802AA21B4004D21B80B4
:100DDE0020E546600874E6254690003AF075460018
:100DEE00E545600874F0254590003AF0754500C25F
:100DFE001B8002C21BE5466003020EA5754600E588
:100E0E0099B4FF03754501E599B4FE03754502E5F6
:100E1E0099B4FD03754503E599B4FC03754504E5E6
:100E2E0099B4FA03754505E599B4FB03754601E5DA
:100E3E0099B4F903754604E599D394E54007E5990D
:100E4E00C394F0400280168599477546027E017F55
:100E5E0000E547C394E6124E858E2E8F2F75310016
:100E6E00753000E599D394C74007E599C394E640E1
:100E7E0002801F85994775460374E5C39547F52F84
:100E8E00752E00AE2EAF2F904BFB124E46783012C1
:100E9E004EC0D2990211CAE546B401028003020F78
:100EAE007DAE30AF31900065124EACE599F07830E2
:100EBE00124EE2AE30AF31EFB40106EEB40702804F
:100ECE0003020F7D900765E0B43C028003020F67BA
:100EDE00C29C1205881202B1900061E09000D4F01D
:100EEE00900062E090008BF0900063E090008CF038
:100EFE00A2154032754F01E54FD394075026E54FAA
:100F0E009007A5F8E4F0E8A3F074AA900032F0126E
:100F1E002DDB7464F509750800122DAF784F74013E
:100F2E0026F650D38030754F08E54FD3940E5026D9
:100F3E00E54F9007A5F8E4F0E8A3F074AA9000320C
:100F4E00F0122DDB7464F509750800122DAF784F81
:100F5E00740126F650D31231AF74C89007A5F8E489
:100F6E00F0E8A3F0D29C7546007545007599FBE537
:100F7E0046B402028003021027E531453070068523
:100F8E00992D752C00AE30AF3174016F4E701BACC5
:100F9E002CAD2DAA2EAB2FED2BFBEC3AFA8A068B3D
:100FAE0007900065124EACE599F07830124EE2AE25
:100FBE0030AF3174026F4E7060AC2CAD2D740D6D70
:100FCE004C702C74639007A5F8E4F0E8A3F074ABB2
:100FDE00900032F0900072E090004FF012311490B9
:100FEE000032E4F074C89007A5F8E4F0E8A3F0E549
:100FFE0047B4E619AE2CAF2D74566F4E600C744884
:10100E006F4E600674666F4E70031205881202B141
:10101E00854799754600754500E546B4033FAE30E9
:10102E00AF31900065124EACE599F07830124EE279
:10103E00AE30AF31AC2EAD2F8F028E038C068D07E6
:10104E00904C37124E46E493F9740193FEEAD39E08
:10105E00EB994009854799754600754500E546B4FC
:10106E00040280030211CAAE30AF31900065124EF9
:10107E00ACE599F07830124EE2AE30AF31EFB400FD
:10108E0006EEB4010280030211CA120588900048D0
:10109E00E075F002A4FFAEF08F4FEF900065124E98
:1010AE00B7EFFCE0FDEC900068124EB7EDFCE0FDF2
:1010BE00EC2DFC900048E0B5040280030211BB0F3A
:1010CE00EF900065124EB7E54FFFE0FCEF90006920
:1010DE00124EB7ECFFE0FCEFC39CFF900048E0B56A
:1010EE00070280030211BBE54F900067124EB7E571
:1010FE004FFFE0FCEF90006A124EB7ECFFE0FCEF02
:10110E002CFF900048E0B5070280030211BBE54FAB
:10111E0090006B124EB7FFE0FCEF900048E0F40435
:10112E002C90004FF0E54F90006C124EB7FFE0FC94
:10113E00EF900048E0F4042C900050F0E54F900042
:10114E006D124EB7FFE0FCEF900048E0F4042C90D7
:10115E000051F0E54F90006E124EB7FFE0FCEF909D
:10116E000048E0F4042C9007A5F8E4F0E8A3F0742E
:10117E00AB900032F01231147464F5097508001248
:10118E002DAF9007A5124E931231147464F50975A4
:10119E000800122DAF9007A5124E931231147599B7
:1011AE00F97464F509750800122DAF80FE7599FF6C
:1011BE007464F509750800122DAF80FEE5456006D2
:1011CE00A299B3B3400302134AC299E545B4011F75
:1011DE00AE30AF3190003E124EACE0F59978301241
:1011EE004EE2AE30AF3174116F4E7003754500E5AF
:1011FE0045B40203854999E545B4031DAE30AF31C0
:10120E00900065124EACE0F599EFB40107EEB4070D
:10121E00037545007830124EE2E545B404028003B2
:10122E0002130CE53145307003852599AE30AF3190
:10123E0074016F4E7003853799AE30AF3174026F03
:10124E004E7003853999AE30AF3174036F4E700313
:10125E00853D99AE30AF3174046F4E7003853F9962
:10126E00AE30AF3174056F4E7003854099AE30AF1E
:10127E003174066F4E7003854199AE30AF317407ED
:10128E006F4E7003854299AE30AF3174086F4E7059
:10129E0006900017E0F599AE30AF3174096F4E70BD
:1012AE0017A21CB340077599FAC21C800B90003A26
:1012BE00E0F59990003AE4F0AE30AF31740A6F4E1B
:1012CE007003854399AE30AF31740B6F4E7003854A
:1012DE003E99AE30AF31740C6F4E7003854499AEAB
:1012EE0030AF31740D6F4E70037599FC7830124E1D
:1012FE00E2AE30AF31740E6F4E7003754500E545AA
:10130E00B40539900040E0D394044010AE30AF31B4
:10131E009049A3124EACE493F599800EAE30AF31E6
:10132E00904A8D124EACE493F599AE30AF3174E91C
:10133E006F4E70037545007830124EE2E54664013B
:10134E006005E546B40403020DBCC28E7E107F001C
:10135E00E53C124E85E58D75F010A4FDACF0EF2D39
:10136E00FDEE3CFCE58B75F01084FF7E00ED2FFF4B
:10137E00EC3EFE8E268F27D28E900092E060569025
:10138E000018124E93900018E0FCA3E0FD90001A96
:10139E00E0FAA3E0FBEDB5033CECB50238B214A2C3
:1013AE0006B34013A214B34008E5B54404F5B58066
:1013BE0006E5B554FBF5B590001AE0FEA3E0FF90EC
:1013CE00001CE0FCA3E0FDEF2DFDEE3CFC90001AAE
:1013DE00ECF0A3EDF090009FE0600990009FE0C359
:1013EE0094034002806F1246E9A206B350099000A2
:1013FE005DE0C3944640028006900089E0F56AE500
:10140E006A75F005A4FFAEF09007A7EEF0A3EFF01B
:10141E00900076E0C395394007E537C395385007FD
:10142E009007A7E4F0A3F0AE57AF589007A7E0FCE3
:10143E00A3E0FDEFD39DEE9C4004C2A1800B900073
:10144E005DE0C394645002D2A190009FE0B4020507
:10145E00A2A1B392A290009FE0B4031C124804AE66
:10146E0057AF589007A7E0FCA3E0FDEFD39DEE9C8D
:10147E004004D2A18002C2A190007AE06009A2B31A
:10148E00300801B3B340028039A2B3300801B34033
:10149E0031A2B3300A01B3401C9000ADE0B4030694
:1014AE00A216B3B340028006740590003AF0D2162D
:1014BE00A20AB39208A20AB330B301B34004A20A3F
:1014CE009208A2B6300701B35003021A03A2B63037
:1014DE000701B35003021A03A2B6300901B3500339
:1014EE00021958754900900092E07013A209B3409A
:1014FE0008E5B554FBF5B58006E5B54404F5B5052C
:10150E0036A20BB3B35013AE26AF27900008E0FC03
:10151E00A3E0FDEDC39FEC9E4003021623E548B405
:10152E000330E536B42305754801801FA21DB34074
:10153E001AE536C39423500690003A7401F0E5364E
:10154E00D394234006740290003AF0753601D21DF2
:10155E00805AE548B40206754801753623E536B45F
:10156E002305753601804590003AE07030E536C3AC
:10157E009423500690003A7401F0E536D39423403C
:10158E0006740290003AF0E536C394235002D21A44
:10159E00E536D394234002D21AC296C2959000AF7C
:1015AE00E0B402051205888003753601AE28AF2916
:1015BE00AC26AD27EF2DFDEE3CFC74028C068D079C
:1015CE00124E778E288F29900092E0603F9000187F
:1015DE00E0FCA3E0FD900092E0FF124E6774018CD8
:1015EE00068D07124E7790001CEEF0A3EFF09000E0
:1015FE001CE0F8A3E090001AC8F0A3C8F090001801
:10160E00E4F0A3F0C214E5B554FBF5B5A21AB3404D
:10161E0002C21A802BAE28AF29AC26AD27EF2DFDC6
:10162E00EE3CFC74018C068D07124E778E288F29A6
:10163E00AC26AD27EDD39488EC94134003120588A5
:10164E00E536B42312740390003AF0D21A9000AF2C
:10165E00E0B40203120588AE2AAF2BAC26AD27EFFD
:10166E002DFDEE3CFC8C2A8D2BAE26AF27EFD39DA5
:10167E00EE9C4011900010E0FAA3E0FBEBC394E85F
:10168E00EA940340028006900010124E9390000CD4
:10169E00E0FEA3E0FFAC26AD27EF2DFDEE3CFC9067
:1016AE00000CECF0A3EDF09000AFE0B40218AE2603
:1016BE00AF277405124E857401124E77900008EE16
:1016CE00F0A3EFF08011AE26AF277402124E859074
:1016DE000008EEF0A3EFF0C28E758D00758B0075CD
:1016EE003C00752701752600D28EE536240875F06C
:1016FE000984AFF07E00EF4E707590000CE0F8A3F9
:10170E00E090000AC8F0A3C8F090000AE0FEA3E043
:10171E00FFEF4E600B7C7B7D89124D658E248F25ED
:10172E0090000CE4F0A3F0AE24AF257428BE0003A5
:10173E009F5010E53B2FFF50010E7401124E778E15
:10174E00248F2585253B9000B6E0A824B8000DD344
:10175E0095254008E525900037F080099000B6E009
:10176E0014900037F0E5486006752500752400904A
:10177E0000ADE0B4030890002EE0653660028026CE
:10178E00A216B34004D2178002B21790007AE0601E
:10179E000BA216B35006A217B3B340028006740410
:1017AE0090003AF0C216E536640B6005E536B41DBE
:1017BE000990009FE060031243F1900033E065361C
:1017CE006007900034E0B53603754A00A20CB350A2
:1017DE0006A20BB3B340030218C090006BE0B40135
:1017EE005AE53F75F00584FF7E00900565124EACFC
:1017FE00E0F533753200AE32AF33900069E0124E31
:10180E008574648E048F05FF124E6774C18C068D2D
:10181E0007124E858E348F3590000EE0FEA3E0FF4A
:10182E00AC32AD3312000374648E048F05FF124E7A
:10183E006790000EECF0A3EDF0800F900069E0755C
:10184E00F0C1A4FFAEF08E348F35E539C394CC5081
:10185E0006900069E07002805785F94F85FA507E38
:10186E00017F00E550124E85E54F2FFF50010E8E81
:10187E00328F33AC34AD35EF2DFDEE3CFC8C348D18
:10188E0035D293D294E535F5FBE534F5FCE535F527
:10189E00E9E534F5EA9000ADE0B40314D291D292AA
:1018AE00E535F5EBE534F5ECE535F5EDE534F5EE3E
:1018BE00D20CE548B40106E536640B6002800F7564
:1018CE004B0190003D7401F0E5B54401F5B5E548D6
:1018DE0070739000B2E0600D9000B9E0A824B800DB
:1018EE00069525400280329000B2E0B402179000B7
:1018FE002CE06536600790002DE0B53603754B037E
:10190E00754400800CC200754400900016E4F0A3EC
:10191E00F0740990003AF0802C90002CE06536604F
:10192E000790002DE0B53603754B0190002CE0B505
:10193E00360690003D7401F090002DE0B536067429
:10194E000290003DF0A209B39207A209B330B6018E
:10195E00B35003021A03754901900092E07013A26E
:10196E0009B34008E5B54404F5B58006E5B554FB6A
:10197E00F5B5A2099207E536D3944A4014D20BE589
:10198E0036D3946D400B740390003AF0D21A75362C
:10199E00469000BAE0B40107E542C39414400280B9
:1019AE0003120588744690005DF0E542C3944150E1
:1019BE0009740E90003AF0120588900044E0FE90F3
:1019CE000040E004C39E4009900040E0D3940640DE
:1019DE000974FB90003AF0120588900049E06015FA
:1019EE00900049E0FE900043E06E600974FE9000A6
:1019FE003AF0120588A21AB34004C296C295A20EFE
:101A0E00B3B3500890002EE065366003021AEBA2C5
:101A1E0002B35006A200B3B34003021AE79000AD22
:101A2E00E0B403028003021ABCA206B34067A217F9
:101A3E00B3402D1201A2E535F5FBE534F5FCD2934A
:101A4E00A203B34002D2879000CBE0B40210120181
:101A5E00CFE535F5FBE534F5FC75A700D28780336D
:101A6E001201A2E535F5EBE534F5ECD291A203B304
:101A7E004006E5B54410F5B59000CBE0B402141263
:101A8E0001CFE535F5EBE534F5EC75A700E5B5448A
:101A9E0010F5B580171201A2E535F5FBE534F5FC1E
:101AAE00E535F5EBE534F5ECD293D291802B1201AE
:101ABE00A2E535F5FBE534F5FCD293A203B3400263
:101ACE00D2879000CBE0B402101201CFE535F5FBC2
:101ADE00E534F5FC75A700D287C20ED20FA20FB364
:101AEE00B3500890002FE065366003021BCAA202B5
:101AFE00B35006A200B3B34003021BC69000ADE084
:101B0E00B403028003021B9BA206B34067A217B365
:101B1E00402D1201A2E535F5E9E534F5EAD294A29D
:101B2E0003B34002D2909000CBE0B402101201CF6A
:101B3E00E535F5E9E534F5EA75A700D29080331264
:101B4E0001A2E535F5EDE534F5EED292A203B340F0
:101B5E0006E5B54420F5B59000CBE0B402141201B1
:101B6E00CFE535F5EDE534F5EE75A700E5B5442086
:101B7E00F5B580171201A2E535F5E9E534F5EAE58C
:101B8E0035F5EDE534F5EED294D292802B1201A20A
:101B9E00E535F5E9E534F5EAD294A203B34002D275
:101BAE00909000CBE0B402101201CFE535F5E9E5D7
:101BBE0034F5EA75A700D290D20EC20FE54BB408E9
:101BCE0016123D20A20EB35005A20FB340028004A0
:101BDE00D20ED20F754B1EE54BB40706123AD875CE
:101BEE004B08E54BB4063D90000EE0FEA3E0FFEF80
:101BFE004E6006A206B3B340028023AE51AF5290A0
:101C0E00000EE0FCA3E0FDEF2DFDEE3CFC8C518DB3
:101C1E0052E536D39412500690000E120039123847
:101C2E00AA754B07E54BB4050612370A754B06E548
:101C3E004BB404289000A0E0902D91F82828731240
:101C4E00339E801212339E800D12354C8008123551
:061C5E00FE80031235FEBA
:0F2D9100021C4D021C52021C57021C5C021C61EA
:101C640012009E754B05E54BB403028003021D4A26
:101C74001245E79000A0E0D39402403F900074E046
:101C84002403A824B8000495255009900076E0D3D5
:101C9400953950028008D202740890003AF09000FE
:101CA40074E0A824B80005D39525500B900076E085
:101CB4002403C395395002C2028039900074E02491
:101CC40003A824B8000495255007E537C395384088
:101CD400028008D202740890003AF0900074E0A8E0
:101CE40024B80005D395255009E538240FC395374A
:101CF4005002C2029000BAE07007E542C394144057
:101D0400028002D202A2024005754B04800A754B80
:101D14001E900016E4F0A3F0A206B34029E53F7537
:101D2400F00584FF7E00900565124EACE0C3946913
:101D34005005124426800F90079FE0F8A3E0900717
:101D44009DC8F0A3C8F0E54BB40A028003021E0C40
:101D5400900026E0C394465008C29674469000262C
:101D6400F0900030E0B4011DE559240AF5599007BC
:101D7400A1E0FEA3E0FF740A2FFF50010E9007A11B
:101D8400EEF0A3EFF0900030E0B4021DE559241406
:101D9400F5599007A1E0FEA3E0FF74142FFF500152
:101DA4000E9007A1EEF0A3EFF08559337532009041
:101DB400002CE0F54F12021AE535900026F0900051
:101DC40004E532F0A3E533F0E54F900027F0C211AB
:101DD4009007A1E0F532A3E0F53390002CE0F54F35
:101DE40012021AE535900024F0900000E532F0A3C9
:101DF400E533F0E54F900025F0C210E548B4010545
:101E0400754B0B8003754B03900024E0B5360280BC
:101E140003021EAEA2104072900000E0FEA3E0FF99
:101E2400EF4E6021AE28AF29900000E0FCA3E0FD56
:101E3400120003740A8E048F05FF124E679000008F
:101E4400ECF0A3EDF0900025E0601A900000E0FEB5
:101E5400A3E0FFAC28AD29EF2DFDEE3CFC90000083
:101E6400ECF0A3EDF0900025E0D39401401A90002B
:101E740000E0FEA3E0FFAC28AD29EF2DFDEE3CFC15
:101E8400900000ECF0A3EDF0D210AE26AF27900046
:101E940000E0FCA3E0FDEFC39DEE9C400D1206485C
:101EA400D296C21074C8900024F0A210B3B35007A5
:101EB400900024E0B53602800D120648D29674C80C
:101EC400900024F0C210900026E0B5360280030290
:101ED4001F69A2114072900004E0FEA3E0FFEF4EE0
:101EE4006021AE28AF29900004E0FCA3E0FD1200BD
:101EF40003740A8E048F05FF124E67900004ECF001
:101F0400A3EDF0900027E0601A900004E0FEA3E047
:101F1400FFAC28AD29EF2DFDEE3CFC900004ECF065
:101F2400A3EDF0900027E0D39401401A900004E060
:101F3400FEA3E0FFAC28AD29EF2DFDEE3CFC9000A4
:101F440004ECF0A3EDF0D211AE26AF27900004E02C
:101F5400FCA3E0FDEFC39DEE9C400AC2967446903C
:101F64000026F0C211A211B3B35007900026E0B5C9
:101F74003602800AC2967446900026F0C211E54BE0
:101F8400B40B02800302204D90002AE0C394465013
:101F9400139000BBE0B40104C2968002C29574465B
:101FA40090002AF0900031E0B4011DE559240AF5AF
:101FB400599007A1E0FEA3E0FF740A2FFF50010E21
:101FC4009007A1EEF0A3EFF0900031E0B4021DE51C
:101FD400592414F5599007A1E0FEA3E0FF74142FCF
:101FE400FF50010E9007A1EEF0A3EFF08559337571
:101FF400320090002DE0F54F12021AE53590002AC8
:10200400F0900006E532F0A3E533F0E54F90002BA5
:10201400F0C2139007A1E0F532A3E0F53390002D50
:10202400E0F54F12021AE535900028F0900002E521
:1020340032F0A3E533F0E54F900029F0C212E548F1
:10204400B40103754800754B03900028E0B53602CF
:1020540080030220FAA2124072900002E0FEA3E084
:10206400FFEF4E6021AE28AF29900002E0FCA3E010
:10207400FD120003740A8E048F05FF124E67900050
:1020840002ECF0A3EDF0900029E0601A900002E069
:10209400FEA3E0FFAC28AD29EF2DFDEE3CFC900043
:1020A40002ECF0A3EDF0900029E0D39401401A90E3
:1020B4000002E0FEA3E0FFAC28AD29EF2DFDEE3CCD
:1020C400FC900002ECF0A3EDF0D212AE26AF279004
:1020D4000002E0FCA3E0FDEFC39DEE9C4018120655
:1020E400489000BBE0B40104D2968002D295C2129B
:1020F40074C8900028F0A212B3B35007900028E0EF
:10210400B5360280181206489000BBE0B40104D230
:10211400968002D29574C8900028F0C21290002ACA
:10212400E0B5360280030221CBA213407290000670
:10213400E0FEA3E0FFEF4E6021AE28AF2990000639
:10214400E0FCA3E0FD120003740A8E048F05FF1265
:102154004E67900006ECF0A3EDF090002BE0601ABF
:10216400900006E0FEA3E0FFAC28AD29EF2DFDEEC4
:102174003CFC900006ECF0A3EDF090002BE0D3942F
:1021840001401A900006E0FEA3E0FFAC28AD29EF61
:102194002DFDEE3CFC900006ECF0A3EDF0D213AE66
:1021A40026AF27900006E0FCA3E0FDEFC39DEE9C64
:1021B40040159000BBE0B40104C2968002C295743D
:1021C4004690002AF0C213A213B3B3500790002A1A
:1021D400E0B5360280159000BBE0B40104C29680DD
:1021E40002C295744690002AF0C213E54BB4020271
:1021F40080030222951241891242A090079DE0FEBD
:10220400A3E0FF740A124E8590000AE0FCA3E0FDEF
:1022140074098F02FF124E678D078C038E048A05A2
:102224008B06124D659007A1EEF0A3EFF09000BB72
:10223400E0B401087478BE00059F4002800D7478F4
:102244009007A1F8E4F0E8A3F0801B9007A1E0FE5A
:10225400A3E0FF74F0BE00039F500B74F09007A13D
:10226400F8E4F0E8A3F09007A1E0FEA3E0FFE5594D
:102274002FFF50010E9007A1EEF0A3EFF090003D68
:10228400E0B40103754B0A90003DE0B40203754BC2
:102294000BE54BB401259000D2E0902DA0F828283E
:1022A40073123F278012123F27800D123FB180081E
:0822B40012405D800312405D41
:0F2DA0000222A50222AA0222AF0222B40222B905
:1022BC00754B029000BDE0B4020280030223D7905C
:1022CC000060E0D3953E5064900060E0F404253E3D
:1022DC00FE9000C0E08E00F5F0E884FF7E008F4F8A
:1022EC00EFC39410500CEF854FF0A4FDACF08D4F64
:1022FC008003754FFF900060E0D3954F400B90002A
:10230C0060E0C3954FF54C8003754C009000DBE00A
:10231C00D3954C40069000DBE0F54C9000DCE0C31C
:10232C00954C50069000DCE0F54C8071900060E01C
:10233C00C3953EFE9000C0E08E00F5F0E884FF7E71
:10234C00008F4FEFC39410500CEF854FF0A4FDACF1
:10235C00F08D4F8003754FFF854F33753200900021
:10236C0060E02533FFAE3250010E8E328F3374FF96
:10237C00BE0009D39F400585334C8003754CFF90FC
:10238C0000DBE0D3954C40069000DBE0F54C900070
:10239C00DCE0C3954C50069000DCE0F54CA206B393
:1023AC00B350099000C8E0D3954D5002800A7407D1
:1023BC0090003AF0C297801375A710E5CDC3954CE9
:1023CC004004C2978002D29775A700A204B34015AF
:1023DC0075A710E5CDC394BF4004C2908002D29083
:1023EC0075A700801375A710E5CDC394404004C2B7
:1023FC00908002D29075A700A205B3401575A71066
:10240C00E5CDC394BF4004C2878002D28775A70074
:10241C00801375A710E5CDC394404004C287800299
:10242C00D28775A700E54AC394094003022B6CA21E
:10243C00EDB35003022B6CC2EDE54A60030225E0BC
:10244C0090006EE070030225CF9000A4E0B401026E
:10245C00800302252F900033E0B53602800302255D
:10246C002C7E017F00E5BE124E85E5BD2FFF50018D
:10247C000E8E328F3390006EE0B401187410124E31
:10248C0085900064E08E048F05FF124E67ED90007E
:10249C0035F0802CAE32AF337410124E8590006440
:1024AC00E08E048F05FF124E67900035E02DFD5035
:1024BC00010C74018C068D07124E77EF900035F0ED
:1024CC00E54360089000CAE064026002802190003D
:1024DC00CCE0B4011A900035E075F0E7A4FFAEF043
:1024EC00E5438E048F05FF124E67ED900035F0909A
:1024FC000035E0FE900036E0D39E4004D2188002F6
:10250C00B218900035E0900036F09000A0E0640125
:10251C006006A218B3B340028006900035E0F53790
:10252C000225CDD2187E017F00E5BE124E85E5BD99
:10253C002FFF50010E8E328F3390006EE0B40118D5
:10254C007410124E85900064E08E048F05FF124EBD
:10255C0067ED900035F0802CAE32AF337410124E14
:10256C0085900064E08E048F05FF124E6790003555
:10257C00E02DFD50010C74018C068D07124E77EF87
:10258C00900035F0E54360089000CAE064026002F8
:10259C0080219000CCE0B4011A900035E075F0E792
:1025AC00A4FFAEF0E5438E048F05FF124E67ED904D
:1025BC000035F09000A0E064016006900035E0F575
:1025CC0037800375370090006AE07005754A01800A
:1025DC000375BB18E54AB401028003022782900000
:1025EC006AE070030227717E017F00E5BE124E8502
:1025FC00E5BD2FFF50010E8E328F339000B0E0B44A
:10260C00010F7E0F7FFFAC32AD33124EDA8E328F5C
:10261C00339000D5E0B40245AE32AF33900020E0E9
:10262C00FCA3E0FDEDD39FEC9E400A900020E53228
:10263C00F0A3E533F0AE32AF33900022E0FCA3E020
:10264C00FDEFD39DEE9C400A900022E532F0A3E50D
:10265C0033F0AE32AF337404124E778F399000D50D
:10266C00E0704CAE32AF33900020E0FCA3E0FDEF05
:10267C00D39DEE9C4009124EDA8E328F3380067554
:10268C003300753200AE32AF337410124E859000A9
:10269C0061E08E048F05FF124E678C328D3374000F
:1026AC00D39D74019C400585333980037539FF90A7
:1026BC0000A0E0B40102800302276FA206B3B3505E
:1026CC000E900074E0A824B80005D39525500302A1
:1026DC002764900075E075F019A4FFAEF09000B877
:1026EC00E08E048F05FF124E679000B1E08539F043
:1026FC00A4FFAEF074648D028C038E048F05FF1260
:10270C004E67EA2DFDEB3CFC8C328D33E543600FBC
:10271C009000CAE0B402089000CCE0640160028032
:10272C0017AE32AF3374E7124E85E5438E048F0536
:10273C00FF124E678C328D33900035E0A832B80012
:10274C000AD395334005853337800BA218B3400666
:10275C00900035E0F537800BA218B3400690003599
:10276C00E0F537800375390090006DE07005754A0F
:10277C0002800375BB19E54AB40202800302283DAE
:10278C0090006DE0700302282CE536D394124003C0
:10279C0002282A90001EE0FEA3E0FFE53D124ED277
:1027AC0090001EEEF0A3EFF07E017F00E5BE124E0E
:1027BC0085E5BD2FFF50010E8E328F339000DAE08D
:1027CC007013740A124E8574518E048F05FF124ECD
:1027DC00678D3D8019AE32AF33740A124E858F046B
:1027EC008E057E017F95CDCCCD124D658F3DE53D9F
:1027FC00D394644003753D6490001EE0FEA3E0FF9B
:10280C00E53D2FFF50010E90001EEEF0A3EFF0906F
:10281C000071E0048E048F05FF124E678D3D80031E
:10282C00753D329000BDE07005754A03800375BBA1
:10283C0013E54AB4035E9000BDE060477E017F0063
:10284C00E5BE124E85E5BD2FFF50010E8E328F3343
:10285C007404124E778F3E9000BFE0853EF0A4FDCD
:10286C00ACF07464FF124E678D3E9000BEE0853E66
:10287C00F0A4FFAEF074FF8E048F05FF124E678D2F
:10288C004D8003753E0090006BE07005754A048026
:10289C000375BB17E54AB40402800302293E90007D
:1028AC006BE0B4017C7E017F00E5BE124E85E5BD78
:1028BC002FFF50010E7404124E778E328F3390001E
:1028CC0038E06012900038E014904C7393A832B842
:1028DC000006953340028006900038E014F090001A
:1028EC0038E0C394775013900038E004904C739305
:1028FC00A832B80005D3953350028006900038E01A
:10290C0004F0900038E0FE900091E08E0088F0A476
:10291C00FFAEF074648E048F05FF124E678D3F80FE
:10292C0003753F0090006CE07005754A05800375D7
:10293C00BB16E54AB4050280030229D190006CE075
:10294C00B4017C7E017F00E5BE124E85E5BD2FFFF4
:10295C0050010E7404124E778E328F33900039E092
:10296C006012900039E014904CEC93A832B8000639
:10297C00953340028006900039E014F0900039E065
:10298C00C394775013900039E004904CEC93A83228
:10299C00B80005D3953350028006900039E004F05E
:1029AC00900039E0FE900097E08E0088F0A4FFAE16
:1029BC00F074648E048F05FF124E678D4080037592
:1029CC00400075BB1FE54AB406337E017F00E5BEAF
:1029DC00124E85E5BD2FFF50010E8E328F337409D8
:1029EC00124E8574E68E048F05FF124E678D429051
:1029FC000073E07005754A07800375BB15E54AB492
:102A0C0007028003022B13900073E07003022B0269
:102A1C007E017F00E5BE124E85E5BD2FFF50010EF5
:102A2C008E328F337404124E778F41900073E0B462
:102A3C0001159000C7E08541F0A4FFAEF0740712B9
:102A4C004E77EF9007AAF0900073E0B40215900057
:102A5C00C7E08541F0A4FFAEF07407124E77EF90FB
:102A6C0007A9F0900073E0B403028003022B0090DE
:102A7C0000B4E0701CE541C3940A5002D201E54158
:102A8C00D394644002C201900093E090005FF08008
:102A9C0063900093E070349000C7E08541F0A4FF90
:102AAC00AEF074FF8E048F05FF124E67ED90005F41
:102ABC00F0AE24AF25741EBE0006D39F4002D20197
:102ACC00E539D394E54002C2018029E541C3940A5B
:102ADC00500DAE24AF25741EBE0004D39F5002804F
:102AEC0002D201E539D394E54002C201900093E093
:102AFC0090005FF080037541009000CAE07005758E
:102B0C004A08800375BB14E54AB408509000CAE02B
:102B1C0060397E017F00E5BE124E85E5BD2FFF506A
:102B2C00010E8E328F33EFD39421EE940E40057547
:102B3C0043FF8015AE32AF337410124E8574E38EA2
:102B4C00048F05FF124E678D438003754300900080
:102B5C006EE0600575BB1A800375BB18054AD2EC94
:102B6C00AE26AF277410C39F74279E400C90005E56
:102B7C00E0C3943C4003022D8EC20B753646900088
:102B8C00AFE070057548028003754803C293C29488
:102B9C00C291C292C287C290E5B554EFF5B5E5B5C6
:102BAC0054DFF5B5C296C295C2A0C297C2A2C2A10B
:102BBC00E5B5547FF5B5E5B554BFF5B5A219B340ED
:102BCC0008E5B54404F5B58006E5B554FBF5B5A2AA
:102BDC000DB3500EE539D394334007E539C394CC8B
:102BEC004003022C74E5B54401F5B5744690005DC4
:102BFC00F0900069E075F064A4FFAEF08E348F3570
:102C0C007402BE000AD39F400675350275340085E8
:102C1C00F94F85FA507E017F00E550124E85E54F45
:102C2C002FFF50010E8E328F33AC34AD35EF2DFDAE
:102C3C00EE3CFC8C348D35D293D294E535F5FBE526
:102C4C0034F5FCE535F5E9E534F5EA9000ADE0B492
:102C5C000314D291D292E535F5EBE534F5ECE5357C
:102C6C00F5EDE534F5EED20DE539C3941A5002C2F8
:102C7C000D90000874FFF0A374DCF0900090E090CD
:102C8C00000EF8E4F0E8A3F0C210C21274C8900071
:102C9C0024F074C8900028F0C20EC20F7525007580
:102CAC002400753B00C206756B00900016E4F0A37F
:102CBC00F0754B1E90079FE0FEA3E0FF7403124ECD
:102CCC00857401124E7790079DEEF0A3EFF0900003
:102CDC0082E0600512009E8002C204900085E060D4
:102CEC00051245E78002C205C203752B00752A0048
:102CFC00900010E4F0A3F0900071E075F032A4FFA6
:102D0C00AEF090001EEEF0A3EFF090000CE4F0A3F8
:102D1C00F0C21D90005EE0C3943C5010E54AB4092B
:102D2C000990005EE004F0754A00803BE54AB40966
:102D3C0003754A00752700752600758D00758B008C
:102D4C00753C0090005DE0C39464500890005DE019
:102D5C0004F08006746490005DF090005DE0B46453
:102D6C0006E5B554FEF5B590005EE0D3940140073E
:102D7C00E542C3944140028009740E90003AF0126F
:052D8C000588020DBCEA
:104BFB000000010001400160018001A001C001E043
:104C0B0002000300039603B603D603F40400050069
:104C1B0005180530054805600578059005A805C001
:104C2B00060006140628063C066E068C00FF013FA4
:104C3B00015F017F019F01BF01DF01FF02FF0395B0
:104C4B0003B503D503F303FF04FF0517052F054732
:104C5B00055F0577058F05A705BF05FF061306271B
:104C6B00063B066F068B06A9DAD8D7D5D4D2D0CFA0
:104C7B00CDCBC9C7C6C4C2C0BEBCBAB8B5B3B1AF41
:104C8B00ADABA8A6A4A2A09D9B99969492908D8B58
:104C9B0089878482807E7C79777573716F6D6B6980
:104CAB00676563615F5D5B5957565452504F4D4B6F
:104CBB004A4847454442413F3E3C3B3A39373635FB
:104CCB00343231302F2E2D2C2B2A2928272625251F
:104CDB002423222121201F1E1E1D1C1C1B1A1A19E6
:104CEB0019EEECEBEAE9E8E7E5E4E3E1E0DEDDDB36
:104CFB00D9D8D6D4D2D0CECCCAC8C6C3C1BFBCBA01
:104D0B00B7B5B2B0ADABA8A5A3A09D9B989592905B
:104D1B008D8A8785827F7D7A7775726F6D6A6865FC
:104D2B0063615E5C5A575553514F4D4B4947454351
:104D3B0042403E3C3B393836353332312F2E2D2B0A
:104D4B002A292827262524232221201F1E1D1D1C2E
:0A4D5B001B1A1A191818171616155E
:102DAF00750B00750A00AE0AAF0BAC08AD09EDC389
:102DBF009FEC9E401674FF124E5775CF01780B741F
:102DCF000126F6500418E436F650DB22900032E06C
:102DDF00B4AA1C900765E0B43C159007A5E0FEA3CC
:102DEF00E0FFEF4E6009741EBE0004D39F50030234
:102DFF002F0975350075340075F8099007A5E0FEA9
:102E0F00A3E0FF74076F4E6006740E6F4E7006746A
:102E1F003A900765F09007A5E0FEA3E0FF7408BEA7
:102E2F00001ED39F401A7E017F089007A5E0FCA3E8
:102E3F00E0FD1DBDFF011C1200038E328F33801F7A
:102E4F009007A5E0FEA3E0FF7408124ED28F048E08
:102E5F00057E017F08CDCCCD1200038E328F33AEAD
:102E6F0034AF35740CD39F74019E5003022F04A20C
:102E7F00F9B3407EE5354534700375A382AE34AFA8
:102E8F003574016F4E700375A300AE34AF35740205
:102E9F006F4E700D9007A6E075F002A4FDACF08D9B
:102EAF00A3AE34AF3574036F4E700375A300AE3409
:102EBF00AF357403BE00039F5013AC32AD33ED2F0B
:102ECF00FFEC3EFE900061124EACE0F5A3AE34AFC6
:102EDF0035EFB40B09EEB401057414124E57AE342E
:102EEF00AF35EFB40B07EEB4010375F80D7834125C
:102EFF004EE2022E6E900032E4F0227535007534EA
:102F0F000075F8099007A5E0FEA3E0FF7408BE0066
:102F1F001ED39F401A7E017F089007A5E0FCA3E017
:102F2F00FD1DBDFF011C1200038E328F33801F90D9
:102F3F0007A5E0FEA3E0FF7408124ED28F048E05A2
:102F4F007E017F08CDCCCD1200038E328F33AE348D
:102F5F00AF357411D39F74019E500302303AA2F91A
:102F6F00B35003023037E5354534700375A3D2AE45
:102F7F0034AF3574016F4E700375A300AE34AF35A7
:102F8F0074026F4E700D9007A6E075F002A4FDACB1
:102F9F00F08DA3AE34AF3574036F4E700375A3007D
:102FAF00AE34AF3574046F4E700375A300AE34AFFB
:102FBF003574056F4E700375A300AE34AF357406CC
:102FCF006F4E700375A300AE34AF3574076F4E703C
:102FDF000375A300AE34AF3574086F4E700375A33D
:102FEF0000AE34AF357408BE00039F5016AC32AD3F
:102FFF0033ED2FFFEC3EFE90005C124EACE5A3F0DC
:10300F0075A300AE34AF35EFB41009EEB4010574FB
:10301F0014124E57AE34AF35EFB41007EEB40103B0
:10302F0075F80D7834124EE2022F5D22753500755A
:10303F00340075F809AE34AF357417BE0004D39F52
:10304F005003023113A2F9B35003023110E5354595
:10305F0034700375A3D2AE34AF3574016F4E700365
:10306F0075A300AE34AF3574026F4E700D9007A686
:10307F00E075F002A4FDACF08DA3AE34AF35740350
:10308F006F4E700375A300AE34AF3574046F4E707E
:10309F000375A300AE34AF3574056F4E700375A37F
:1030AF0000AE34AF3574066F4E700375A300AE34A7
:1030BF00AF3574076F4E700375A300AE34AF357420
:1030CF00086F4E700375A300AE34AF357408BE00A1
:1030DF00039F500C900046124EACE5A3F075A30071
:1030EF00AE34AF3574166F4E70057414124E57AE62
:1030FF0034AF3574166F4E700375F80D7834124E69
:10310F00E202304422900032E0B4AB02800302317D
:10311F00AE75350075340075F809AE34AF357412DD
:10312F00BE007CD39F4078A2F9B34070E53545349B
:10313F00700375A382AE34AF3574016F4E70037593
:10314F00A300AE34AF3574026F4E700D9007A6E03A
:10315F0075F002A4FDACF08DA3AE34AF3574036FE0
:10316F004E700375A300AE34AF357403BE00039FDA
:10317F00500990004B124EACE0F5A3AE34AF35744E
:10318F00116F4E70057414124E57AE34AF35741163
:10319F006F4E700375F80D7834124EE2023129220A
:1031AF0090003BE4F074649007A5F8E4F0E8A3F016
:1031BF0012303B74C89007A5F8E4F0E8A3F0900034
:1031CF0052E0B4371A90004FE0900046F090005054
:1031DF00E0900047F0900051E0900048F08046905A
:1031EF00003B7401F074659007A5F8E4F0E8A3F0D4
:1031FF0012303B74C89007A5F8E4F0E8A3F09000F4
:10320F0052E0B4371A90004FE0900046F090005013
:10321F00E0900047F0900051E0900048F080067475
:10322F000290003BF090003CE4F074669007A5F824
:10323F00E4F0E8A3F012303B74C89007A5F8E4F06F
:10324F00E8A3F0900051E0B4371290004FE09000E7
:10325F0040F0900050E0900049F0807690003C7470
:10326F0001F074679007A5F8E4F0E8A3F012303B83
:10327F0074C89007A5F8E4F0E8A3F0900051E0B40B
:10328F00371290004FE0900040F0900050E0900017
:10329F0049F0803E740290003CF074689007A5F8E6
:1032AF00E4F0E8A3F012303B74C89007A5F8E4F0FF
:1032BF00E8A3F0900051E0B4371290004FE0900077
:1032CF0040F0900050E0900049F0800674039000A9
:1032DF003CF022E55C2533FFAE3250010E900065C5
:1032EF00124EACE0F55DE55C2533FFAE3250010EBA
:1032FF000FBF00010E900065124EACE0F55E8564C5
:10330F0060E55DB55E05855D5C8041E55ED3955DED
:10331F00401DE55EC3955D855FF0A4FFAEF0E560EF
:10332F008E048F05FF124E67ED255DF55C801DE560
:10333F005DC3955E855FF0A4FFAEF0E5608E048FF0
:10334F0005FF124E67EDF404255DF55C22E55ED3B3
:10335F00955D401DE55EC3955D855FF0A4FFAEF002
:10336F00E5608E048F05FF124E67ED255DF55C80DD
:10337F001DE55DC3955E855FF0A4FFAEF0E5608E41
:10338F00048F05FF124E67EDF404255DF55C22E511
:10339F003775F00484FF7E008F5CE53775F0048489
:1033AF00ADF07C008D5F756404753201753300E5F7
:1033BF005CC3943F50051232E280069001A4E0F501
:1033CF005C855C52755100900037E075F020A4FFCA
:1033DF00AEF09000B6E08E048F05FF124E678D5C45
:1033EF0090009EE0D3953750030234A49000C2E0C2
:1033FF00D395374010ED9001A5124EB7E0F55475F7
:10340F0053000234A190008DE0D395374043E55C23
:10341F009001A5124EB7E0F55DE55C9001C5124E27
:10342F00B7E0F55E9000C2E0F4042537F55F900039
:10343F008DE0FE9000C2E0F4042EF560E55DB55E10
:10344F0005855D5C800312335C855C547553008089
:10345F0041E55C9001C5124EB7E0F55DE55C90016A
:10346F00E5124EB7E0F55E90008DE0F4042537F5D8
:10347F005F90009EE0FE90008DE0F4042EF560E575
:10348F005DB55E05855D5C800312335C855C5475AC
:10349F00530002354B9000C5E0D395375011E55CD2
:1034AF00900225124EB7E0F55475530002354B903C
:1034BF00008EE0D395375043E55C900205124EB76E
:1034CF00E0F55DE55C900225124EB7E0F55E9000E9
:1034DF008EE0F4042537F55F9000C5E0FE90008E76
:1034EF00E0F4042EF560E55DB55E05855D5C800357
:1034FF0012335C855C547553008041E55C9001E5A7
:10350F00124EB7E0F55DE55C900205124EB7E0F59F
:10351F005E90009EE0F4042537F55F90008EE0FE8C
:10352F0090009EE0F4042EF560E55DB55E05855DC7
:10353F005C800312335C855C54755300229000D677
:10354F00E0F561756411753202753300AE24AF2555
:10355F00E56175F00FA4FDACF0EDD39FEC9E40211B
:10356F00E5618E048F05FF124E67ED75F010A4FF15
:10357F00AEF0E53775F01184FD7C00ED2FF562801C
:10358F000EE53775F01184FF7E00EF24F0F56285AC
:10359F00625CE53775F01184AFF07E008F5F1232F9
:1035AF00E2855C63AE24AF259000D6E075F00FA4E2
:1035BF00FDACF0EDD39FEC9E4028753202753310B1
:1035CF0085625C1232E285635D855C5EAE24AF2559
:1035DF00E5618E048F05FF124EA08D5F856160122D
:1035EF00335C855C5275510075546475530022909D
:1035FF0000D6E0F561756411753202753300AE24A3
:10360F00AF25E56175F00FA4FDACF0EDD39FEC9EF7
:10361F004021E5618E048F05FF124E67ED75F010A6
:10362F00A4FFAEF0E53975F01184FD7C00ED2FF5A8
:10363F0062800EE53975F01184FF7E00EF24F0F5FE
:10364F006285625CE53975F01184AFF07E008F5FA3
:10365F001232E2855C63AE24AF259000D6E075F0A0
:10366F000FA4FDACF0EDD39FEC9E40287532027590
:10367F00331085625C1232E285635D855C5EAE2439
:10368F00AF25E5618E048F05FF124EA08D5F85611A
:10369F006012335C855C527551009000A0E0B40459
:1036AF0053E53775F00484FF7E008F5CE53775F0C6
:1036BF000484ADF07C008D5F756404753201753341
:1036CF0000E55CC3943F50051232E280069001A4DE
:1036DF00E0F55CAE51AF52E55C124E8574648E041A
:1036EF008F05FF124E67AE51AF52EF2DFDEE3CFC32
:1036FF008C518D527554647553002290006BE0B459
:10370F000146E53F75F00584FF7E008F5CE53F7550
:10371F00F00584ADF07C008D5F756405753205751D
:10372F003300E55CC3941750051232E28006900512
:10373F007CE0F55CAE53AF54E55C2FFF50010E7487
:10374F0064124ED28E538F5490006CE0B40146E554
:10375F004075F00584FF7E008F5CE54075F00584B1
:10376F00ADF07C008D5F756405753205753348E5E6
:10377F005CC3941750051232E280069005C4E0F541
:10378F005CAE53AF54E55C2FFF50010E7464124EC4
:10379F00D28E538F5490007BE0B40249E542C3941C
:1037AF004175F00584FF7E008F5CE54275F005845E
:1037BF00ADF07C008D5F756405753206753300E5DD
:1037CF005CC3941350051232E28006900678E0F540
:1037DF005CAE53AF54E55C2FFF50010E7464124E74
:1037EF00D28E538F549000BDE0B402028003023892
:1037FF00A9E53775F01584FF7E008F5CE53775F00E
:10380F001584ADF07C008D5F7564157532037533CB
:10381F00F4E55CC3940B50051232E2800690046409
:10382F00E0F55CE55C75F0FFA4FFAEF09000BEE044
:10383F008E048F05FF124E67ED900060F0E53E7528
:10384F00F078A4FFAEF074FF8E048F05FF124E6761
:10385F008C328D3374028C068D07124E778F5CACD1
:10386F0032AD337404FF124EA08D5F756404753250
:10387F000675336EE55CC3941D50051232E2800667
:10388F009006F0E0F55CAE53AF54E55C2FFF5001AE
:10389F000E7464124ED28E538F5422900073E0B484
:1038AF0001179007AAE02554FFAE5350010E900068
:1038BF00C7E0124ED28E538F54900073E0B40316AC
:1038CF00A201B3B3501090005FE0C39405A824B8D1
:1038DF000006952540028010900095E02554FFAE1C
:1038EF005350010E8E538F5490006DE0B40202803E
:1038FF0003023AD7900070E0602FE53FD3941E404B
:10390F0028900010E0FEA3E0FF9000ABE075F003FD
:10391F00A4FDACF0EFD39DEE9C400E9000CFE0A83D
:10392F0024B80005D395255003023AD79000B8E08C
:10393F008537F0A4FFAEF07405124E857407124E52
:10394F00778E328F33900077E0A824B80004952546
:10395F005012900078E075F002A4FDACF0EFC39D1B
:10396F00EE9C4003023AD7E53775F00B84FF7E00DB
:10397F009005F5124EACFEE0FFEE90006FE0FEEF0B
:10398F008E0088F0A4FFAEF074648E048F05FF12D2
:10399F004E678C328D33900037E075F018A4FFAE70
:1039AF00F09000B6E08E048F05FF124E678C068DE7
:1039BF000790060D124EACAE32AF33E0124E857447
:1039CF00648E048F05FF124E678C328D33E53DA850
:1039DF0032B80077D395334072E53DC39533FFE49A
:1039EF009532FE8E328F337428BE00039F500C75B4
:1039FF003328753200740D90003AF0AE32AF339029
:103A0F000070E0124E8574288E048F05FF124E67EA
:103A1F008C328D33AE51AF52740A8E048F05FF1264
:103A2F004E678D068C07AC32AD33CFCECF1200036D
:103A3F00740A8E048F05FF124E678C328D33AE5190
:103A4F00AF52124EDA8E518F52807DE53DA832B8BB
:103A5F00000495335072AE32AF33E53D124ED28E25
:103A6F00328F337428BE00039F500C753328753284
:103A7F0000740D90003AF0AE32AF33900070E01248
:103A8F004E8574288E048F05FF124E678C328D334E
:103A9F00AE51AF52740A8E048F05FF124E678D061A
:103AAF008C07AC32AD33CFCECF120003740A8E0425
:103ABF008F05FF124E678C328D33AE51AF52EF2D03
:103ACF00FDEE3CFC8C518D5222AE51AF52AC53AD3A
:103ADF005412000374648E048F05FF124E678C51CD
:103AEF008D52900068E08C068D07124E8574648E9F
:103AFF00048F05FF124E678C518D52A2064017AEF0
:103B0F0024AF257405BE00039F5002D206E539D3BA
:103B1F0094CC4002D2029000CAE0B402089000CCCC
:103B2F00E0640160028017AE51AF52E543124E853B
:103B3F0074E78E048F05FF124E678C518D529000E3
:103B4F008AE05402601B900081E0A824B80012D3D1
:103B5F009525400DA206B3B35007E539C3949A409B
:103B6F00028028AE5AAF5B90007FE075F002A4FD93
:103B7F00ACF0EF2DFDEE3CFC74022DFD50010CE579
:103B8F0039BC0007D39D400375680185395B755AB1
:103B9F0000E5687003023C2E9000DDE0C39568409D
:103BAF0070E53F75F00584FF7E00900565124EAC01
:103BBF00E0F533753200AE32AF3390008FE0124E26
:103BCF008574648E048F05FF124E678C348D35908B
:103BDF0000DDE004C395688C068D07124E859000BA
:103BEF00DDE08E048F05FF124E678C348D3590000B
:103BFF0080E08C068D07124E85740A8E048F05FFA8
:103C0F00124E67AE51AF52EF2DFDEE3CFC8C518D35
:103C1F005205689000DDE0C3956850037568009009
:103C2F00008AE05401601B90007EE0A824B80012C7
:103C3F00D39525400DA206B3B35007E537C394CCF7
:103C4F004002802590007CE075F003A4FFAEF0E504
:103C5F00652FFF50010E74032FFF50010EE537BE85
:103C6F000007D39F4003756901853765E5697003C8
:103C7F00023D099000DEE0C395694070E53F75F0A5
:103C8F000584FF7E00900565124EACE0F53375326A
:103C9F0000AE32AF3390008FE0124E8574648E0405
:103CAF008F05FF124E678C348D359000DEE004C314
:103CBF0095698C068D07124E859000DEE08E048F7D
:103CCF0005FF124E678C348D3590007DE08C068D8C
:103CDF0007124E85740A8E048F05FF124E67AE5180
:103CEF00AF52EF2DFDEE3CFC8C518D5205699000CB
:103CFF00DEE0C39569500375690090008FE0A8510D
:103D0F00B800049552500990008FE0F5527551009C
:103D1F00229000CBE0B401028003023E2BA206B337
:103D2F005003023E29900096E0B40168AE51AF52A5
:103D3F00AC24AD25120003743C8E048F05FF124E88
:103D4F00679000A6E0BC00109D400D9000A8E0A871
:103D5F0051B8000495525002D203AE51AF52AC2469
:103D6F00AD25120003743C8E048F05FF124E679031
:103D7F0000A6E0C3940ABC0015D39D40119000A883
:103D8F00E0C39405A851B80005D3955250028002A4
:103D9F00C2038068AE51AF52AC24AD25120003743C
:103DAF00788E048F05FF124E679000A6E0BC0010BE
:103DBF009D400D9000A8E0A851B800049552500402
:103DCF00D2038038AE51AF52AC24AD25120003742C
:103DDF00788E048F05FF124E679000A6E0C3940AF9
:103DEF00BC0015D39D40119000A8E0C39405A851C5
:103DFF00B80005D3955250028002C203A203B3400C
:103E0F0019AE51AF529000A7E0124E8574648E0424
:103E1F008F05FF124E678C518D528002C2039000A6
:103E2F00CBE0B40258E53775F00884FF7E008F5C55
:103E3F00E53775F00884ADF07C008D5F756408750B
:103E4F0032017533E0E55CC3943F50051232E280D6
:103E5F0006900264E0F55CE55C75F05EA4FFAEF0E1
:103E6F00740A8E048F05FF124E678C558D5674029F
:103E7F00BC000AD39D4006755602755500A200B3CB
:103E8F004006A202B3B35009900016E4F0A3F080ED
:103E9F0024AE51AF527400D39F74019E400C90001A
:103EAF0016E551F0A3E552F0800B74FF900016F861
:103EBF00E4F0E8A3F09000ADE0D394024006A20630
:103ECF00B3B34002800DAE51AF527402124E858EC5
:103EDF00518F52900096E0B4010DAE51AF52740263
:103EEF00124E858E518F52AE51AF52745E124E8567
:103EFF00740A8E048F05FF124E678C518D52740217
:103F0F00BC000AD39D4006755202755100900014F3
:103F1F00E551F0A3E552F022900037E090036512CF
:103F2F004EB7E0F566756764900037E0FE9000A12C
:103F3F00E0D39E4037E53775F00884FF7E008F5C35
:103F4F00E53775F00884ADF07C008D5F75640875FA
:103F5F003203753396E55CC3941F50051232E2802D
:103F6F000690041AE0F55C855C678035E53775F0DF
:103F7F000884FF7E008F5CE53775F00884ADF07C18
:103F8F00008D5F7564087532037533B6E55CC394B5
:103F9F001F50051232E2800690043AE0F55C855C12
:103FAF0067229000D7E0F56175641175320475339F
:103FBF0000AE24AF25E56175F00FA4FDACF0EDD395
:103FCF009FEC9E4021E5618E048F05FF124E67ED39
:103FDF0075F010A4FFAEF0E53775F01184FD7C008D
:103FEF00ED2FF562800EE53775F01184FF7E00EF3F
:103FFF0024F0F56285625CE53775F01184AFF07ED1
:10400F00008F5F1232E2855C63AE24AF259000D73C
:10401F00E075F00FA4FDACF0EDD39FEC9E4028753A
:10402F00320475331085625C1232E285635D855C04
:10403F005EAE24AF25E5618E048F05FF124EA08D75
:10404F005F85616012335C855C66756764229000E2
:10405F00D7E0F561756411753204753300AE24AF86
:10406F0025E56175F00FA4FDACF0EDD39FEC9E40FC
:10407F0021E5618E048F05FF124E67ED75F010A4D8
:10408F00FFAEF0E53975F01184FD7C00ED2FF56280
:10409F00800EE53975F01184FF7E00EF24F0F56294
:1040AF0085625CE53975F01184AFF07E008F5F1289
:1040BF0032E2855C63AE24AF259000D7E075F00F38
:1040CF00A4FDACF0EDD39FEC9E4028753204753300
:1040DF001085625C1232E285635D855C5EAE24AF53
:1040EF0025E5618E048F05FF124EA08D5F856160FF
:1040FF0012335C855C667567649000D2E0B4047916
:10410F00900037E0FE9000A1E0D39E4037E5377571
:10411F00F00884FF7E008F5CE53775F00884ADF002
:10412F007C008D5F756408753203753396E55CC34B
:10413F00941F50051232E2800690041AE0F55C8558
:10414F005C678035E53775F00884FF7E008F5CE58E
:10415F003775F00884ADF07C008D5F75640875329B
:10416F00037533B6E55CC3941F50051232E2800627
:10417F0090043AE0F55C855C672290006BE0B40137
:10418F003BE53F75F00584FF7E008F5CE53F75F0E2
:10419F000584ADF07C008D5F756405753205753350
:1041AF0018E55CC3941750051232E280069005940F
:1041BF00E0F55CE567255CC39464F56790006CE0FF
:1041CF00B4013BE54075F00584FF7E008F5CE54050
:1041DF0075F00584ADF07C008D5F75640575320553
:1041EF00753360E55CC3941750051232E280069078
:1041FF0005DCE0F55CE567255CC39464F567E5666F
:10420F002567F559900073E0B402109007A9E025D7
:10421F0059FE9000C7E0F4042EF5599000CAE0D380
:10422F0094014040E543C394E7501D74E7C39543A1
:10423F00FE9007ABE08E00F5F0E884FF7E008F5C08
:10424F00E559255CF559801CE543C394E7FE9007BB
:10425F00ABE08E00F5F0E884FF7E008F5CE559C37C
:10426F00955CF559A2064006E5662464F559E559B3
:10427F00D394644009E559C39464F5598003755983
:10428F00009000A3E0C3955950069000A3E0F559A4
:10429F0022D2009000B9E0A824B800049525503B25
:1042AF009000B9E0A824B800049525500375590F64
:1042BF009000B9E004A824B800049525500375595F
:1042CF000A9000B9E02402A824B8000495255005EF
:1042DF00755905C200740990003AF07E017F009075
:1042EF0000A9E0124E859000B8E08E048F05FF12F2
:1042FF004E67E537BC000CD39D4008C200740A908E
:10430F00003AF09000AAE0C3953F500D9000BCE03A
:10431F00A824B80006952540028008C200740B90AF
:10432F00003AF0A2004003755905900073E0B40302
:10433F0006A201B3B34002802B90005FE0C3940547
:10434F00A824B800049525500C900094E0F55974FA
:10435F000C90003AF090005FE0A824B80004952577
:10436F005002C200855944900065E02559FE900027
:10437F0037E075F01E84FC7F00EE2CF5592290007B
:10438F0037E075F00584FF7E008F5C900037E07595
:10439F00F00584ADF07C008D5F7564057532037593
:1043AF0033D69000B6E01475F00584FF7E00E55C0F
:1043BF00BE00039F50051232E2800BE55C90043B78
:1043CF00124EB7E0F55CE55C9007ACF09007ACE0FF
:1043DF00FE9000A5E0C39E50089000A5E09007ACAA
:1043EF00F022E53F75F00584FF7E00900565124EC3
:1043FF00ACE0F56BE56BD394644010E56BC394644C
:10440F0075F00F84FF7E008F6B8003756B0090003B
:10441F0088E0256BF56B2290079FE0FEA3E0FF7409
:10442F0004124E77E537124E85740F8E048F05FFF9
:10443F00124E6790079DECF0A3EDF090007BE0B477
:10444F000262E542C3944175F00584FF7E008F5CE4
:10445F00E54275F00584ADF07C008D5F75640575E0
:10446F003206753314E55CC3941750051232E2809F
:10447F000690068CE0F55C90079DE0FEA3E0FF74CC
:10448F000A8E048F05FF124E67E55C8C068D0712AE
:10449F004E85740A8E048F05FF124E6790079DECB0
:1044AF00F0A3EDF090079DE0FEA3E0FF9007A3E0DF
:1044BF00FCA3E0FDEDD39FEC9E400F9007A3E0F827
:1044CF00A3E090079DC8F0A3C8F022900082E0B44B
:1044DF00010385254F900082E0B402129000B8E0EE
:1044EF008537F0A4FFAEF07408124E778F4F90000F
:1044FF0082E0B4030385394F900082E0B404038552
:10450F003F4F900082E0B4050385404F900082E05A
:10451F00B4060385414F900082E0B4070385424FF4
:10452F00900082E0B4080385434F900082E0B40905
:10453F0003853E4F900082E0B40A03853D4F900003
:10454F0082E0B40B0385444F900082E0B40C0690D8
:10455F000017E0F54F900083E0FE900084E0D39EBB
:10456F00404B900082E0B40418900084E0C3954F54
:10457F005002D204900083E0D3954F4002C20480D2
:10458F002A900083E0C3954F5009900084E0D395A3
:10459F004F50028002D204900083E0D3954F500910
:1045AF00900084E0C3954F5002C204802A9000838C
:1045BF00E0D3954F4009900084E0C3954F400280AF
:1045CF0002C204900083E0C3954F4009900084E03D
:1045DF00D3954F4002D20422900085E0B4010385A9
:1045EF00254F900085E0B402129000B8E08537F0B7
:1045FF00A4FFAEF07408124E778F4F900085E0B491
:10460F00030385394F900085E0B40403853F4F9035
:10461F000085E0B4050385404F900085E0B40603A4
:10462F0085414F900085E0B4070385424F90008588
:10463F00E0B4080385434F900085E0B40903853E3D
:10464F004F900085E0B40A03853D4F900085E0B49C
:10465F000B0385444F900085E0B40C06900017E0E3
:10466F00F54F900086E0FE900087E0D39E4040908B
:10467F000086E0C3954F5009900087E0D3954F50C7
:10468F00028002D205900086E0D3954F500990002A
:10469F0087E0C3954F5002C205900085E0B4010931
:1046AF009000C4E0D3953950028002C205802A9051
:1046BF000086E0D3954F4009900087E0C3954F40A7
:1046CF00028002C205900086E0C3954F400990001A
:1046DF0087E0D3954F4002D20522AE57AF5874F5FD
:1046EF00D39F74019E40087857124EE2024803751B
:1046FF005801755700AE24AF25E56BBE000DD39F53
:10470F00400990009AE0D3956C40028023756C00AD
:10471F00E56BC39525F54F90009DE0D3956A400852
:10472F00E56A254FF56A800690009DE0F56A8002E4
:10473F00056C900076E0D39539401CE537C395386A
:10474F004015AE24AF25E56BBE00039F50099000C6
:10475F009BE0D3956D4002806E9007ADE0A824B822
:10476F00000495255003756F009007ADE0A824B89D
:10477F00000BD395254006E5259007ADF0E56F704A
:10478F0041E525C3956BF54FE54FD3940540037570
:10479F004F0590009CE0C3956A5007E54FC3956A9B
:1047AF0040028009E56AC3954FF56A800690009C28
:1047BF00E0F56A90009CE0D3956A400690009CE07B
:1047CF00F56A756D008002056DE56F7016900076C5
:1047DF00E0C39539500DE56B2405A824B800069564
:1047EF00254002800F900089E0F56A756F0174789B
:1047FF009007ADF022AE57AF5874E9D39F74039E64
:10480F0040087857124EE20249A2755801755700B9
:10481F00756A32A21E402A756A19900089E075F0F8
:10482F0002A4FFAEF0E56CBE0006D39F4002D21E7D
:10483F00056C756F0374789007ADF0756E000249C3
:10484F0091AE24AF25E56B6F4E7003024991E56B76
:10485F00BE000DD39F400990009AE0D3956C4002A3
:10486F00800F756C00E56FC394035003756A198050
:10487F000DE56BC39525F54FE56C254FF56C900055
:10488F0076E0D39539400E9007ADE0A824B8000725
:10489F00D395254002800C056E900089E0B56E031C
:1048AF00756F00E56FB40306A206B3B34002800A2A
:1048BF00056EE56EB43C03756F02E56FB402299087
:1048CF0007ADE0A824B8000ED395254009E5259043
:1048DF0007ADF0756E00900076E0C39539500975FD
:1048EF006E0074789007ADF0E56F705A900076E027
:1048FF00D39539401CE537D395384015AE24AF25F5
:10490F00E56BBE00039F500990009BE0D3956D406F
:10491F00028008756D00756A4B8028E525C3956B7D
:10492F00F54FE54FD394054003754F05900076E0A2
:10493F00D395394008E56D254FF56D8006E56D245B
:10494F0006F56D756E00E56F7016900076E0C395F5
:10495F0039500DE56B2405A824B8000695254002B3
:10496F008003756F01E56FB40118756A19056E90B4
:10497F000089E0B56E06756F02756E00747890074A
:10498F00ADF0E56A75F00AA4FFAEF09007A7EEF060
:04499F00A3EFF02270
:094EB7002582F5825002058322D8
:0F008C0025E050020583258250020583F582226C
:104E4600EF2F500205832582F582E5833E2EF583FA
:014E56002239
:104ED200CFC39FFF50011E22C3EF9DFFEE9CFE2217
:094EC000E493F608740193F62254
:084EE2000806B60002180622C2
:0D4E9300A3E004F07006120049E004F022D4
:0E003900A3E014F0B4FF06120049E014F02218
:0E4E7700048007C3CE13CECF13CFD5E0F622B2
:104D6500BC000FBE0008ED8FF084FFADF022E4FE1D
:104D7500FF22BE000DEF60FE54F0606F20E70302D6
:104D85004E1BEAC0E0EBC0E078017A0075F001EE59
:104D950020E710EF25E0FFEE33FE0AC5F023C5F04E
:104DA50030E7F0EA5407F9096A7A007B00600108E8
:104DB500C3EC9E40167004ED9F4010ED9FFDEC9EE8
:104DC500FCE5F0CA4ACA03F5F08005E5F003F5F005
:104DD500C3EE13FEEF13FFD9D77908CACBCAD8D0D3
:104DE500EAFEEBFFD0E0FBD0E0FA22EC8FF084FC8A
:104DF500ED54F045F0C48FF084FEEDC454F045F059
:104E0500C48FF084FDEEC4FE54F02DFFEE540F3C2C
:104E1500FEADF07C0022790078008FF0EC7E082052
:104E2500E70DC3CD33CD33C933C9C833C8DEF084EC
:104E350049F9E5F08FF0BE00E6FD7C00E9FFE8FEEC
:014E4500224A
:0E4E8500F88FF0A4FFE5F0CE88F0A42EFE22F8
:10000300EF8DF0A4F9A8F0EF8CF0A428F8EE8DF0B2
:06001300A428FEE9FF2213
:104E5700600D782B024E61007830D8FED5E0F8223D
:104E6700EEC0E07E00124D65EFFDEEFCD0E0FE22C5
:0C4EA000EEC0E07E00124D65D0E0FE2266
:03001B0002001EC2
:0300530002005652
:03009B00020071EF
:03000000024EC9E4
:094EC90075817075D00002072A02
:0B4EAC00E5822FF582E5833EF58322AE
:0A0049000582D5820215831582227C
:10001E00C0E0C0F0C083C082C0D075D00012067D93
:0B002E00D0D0D082D083D0F0D0E032E0
:10005600C0E0C0F0C083C082C0D075D00012068058
:10006600D0D0D082D083D0F0D0E032C0E0C0F0C093
:1000760083C082C0D075D0001206F9D0D0D082D00D
:0600860083D0F0D0E0324F
:00000001FF
